:020000040000FA
:060000002DEF06F01200D6
:060800002DEF06F01200CE
:02082A000000CC
:04082C00D9CFE6FF3B
:10083000E1CFD9FF020EE126DE6ADD6ADECF00F0ED
:10084000DDCF01F0FD0EDBCF02F0FE0EDBCF03F0BB
:1008500001500318E8AE02D0033404D00250005C0B
:10086000035001580AE2010EE66E3BEC06F0E55239
:10087000DF2A010E01E3DB2AE1D7020EE15C02E28E
:10088000E16AE552E16EE552E7CFD9FF1200D9CF18
:10089000E6FFE1CFD9FF040EE126DE6ADE6ADE6AFA
:1008A000DD6ADD52DD52FB0EDBCF00F0FC0EDBCF4C
:1008B00001F0FD0EDBCF02F0FE0EDBCF03F0D9CF4F
:1008C000E9FFDACFEAFF030EEB500318E8AE02D0DF
:1008D000033408D00050EE5C0150EE580250EE5840
:1008E0000350EE580FE20C0EE66E0DEC06F0E552EA
:1008F000D9CFE9FFDACFEAFFEE2A000EEE22EE2290
:10090000EE22D1D7040EE15C02E2E16AE552E16E2B
:10091000E552E7CFD9FF12000F0EC16E936A300E79
:10092000926E0F0E946E1200D9CFE6FFE1CFD9FF81
:10093000020EE1268250020B01E0010E080DF3CFFA
:1009400002F08250010B040DF3CF01F08050200B18
:1009500001E0010EE824006E8050100B01E0010E52
:10096000002401240224DE6EDD6ADECF00F0DDCF3C
:1009700001F000C0F3FF01C0F4FF020EE15C03E2EE
:1009800000D0E16AE552E16EE552E7CFD9FF1200EF
:1009900080920A0EE66EE66A49DFE552E5528084EF
:1009A0000A0EE66EE66A42DFE552E55280940A0ED0
:1009B000E66EE66A3BDFE552E552120080820A0EDF
:1009C000E66EE66A33DFE552E55280840A0EE66E93
:1009D000E66A2CDFE552E55280940A0EE66EE66A7E
:1009E00025DFE552E5521200380E816ED1DF050E8B
:1009F000E66EE66AE66AE66A4ADFE552E552E552E5
:100A0000E552010E816EC4DF050EE66EE66AE66A07
:100A1000E66A3DDFE552E552E552E5520D0E816E84
:100A2000B7DF050EE66EE66AE66AE66A30DFE55293
:100A3000E552E552E552060E816EAADF050EE66E1E
:100A4000E66AE66AE66A23DFE552E552E552E552D8
:100A50001200010E816E9CDF050EE66EE66AE66A04
:100A6000E66A15DFE552E552E552E5521200D9CFAC
:100A7000E6FFE1CFD9FF020E816E8ADF0A0EE66E35
:100A8000E66AE66AE66A03DFE552E552E552E552B8
:100A9000FD0EDBCFE6FFFE0EDB50280DF350E552D6
:100AA000E724E76EFE0EE7CFDBFFFD0EDB6AFE0EEE
:100AB000DB50F36EFD0EDBCFF4FFF350F45C0CE281
:100AC000140E816E65DF010EE66EE66AAFDEE5525A
:100AD000E552FD0EDB2AEBD7E552E7CFD9FF120036
:100AE000D9CFE6FFE1CFD9FFFE0EDB50816E66DF86
:100AF0000A0EE66EE66A9ADEE552E552E552E7CF67
:100B0000D9FF1200D9CFE6FFE1CFD9FFFD0EDBCF31
:100B1000E9FFFE0EDBCFEAFFEF500EE0FD0EDBCF6C
:100B2000E9FFDB2AFE0EDBCFEAFF01E3DB2AEF5011
:100B3000E66ED6DFE552EAD7E552E7CFD9FF1200DD
:100B4000EBDEF2DEF350816E8080E80EE66E030E7F
:100B5000E66EE66AE66A9BDEE552E552E552E5524C
:100B60008090E80EE66E030EE66EE66AE66A8FDEB9
:0C0B7000E552E552E552E552E4D71200D0
:040B7C002A0EF66ED9
:100B8000080EF76E000EF86E02010900F550056FB1
:100B90000900F550066F03E1056701D03DD009005B
:100BA000F550006F0900F550016F0900F550026F14
:100BB00009000900F550E96E0900F550EA6E0900D8
:100BC00009000900F550036F0900F550046F090092
:100BD0000900F6CF07F2F7CF08F2F8CF09F200C20A
:100BE000F6FF01C2F7FF02C2F8FF0201035302E160
:100BF000045307E00900F550EE6E0307F8E204071E
:100C0000F9D707C2F6FF08C2F7FF09C2F8FF0201D1
:0A0C10000507000E065BBFD71200B7
:060C1A00FF0EE350066E20
:100C2000480E01D04C0EE76EE72EFED7E76AE72E9E
:0A0C3000FED7062EF7D700001200D1
:060C3A00000EF36E00EE57
:100C400000F0080E01D81200EA6002D0EE6AFCD76C
:0A0C5000F350E9601200EE6AFCD7D1
:060C5A0012EE40F022EE54
:100C600040F0F86A059CBEEC05F046EC06F0A0ECFE
:060C700005F0FBD71200A5
:0A0C7600FF0EE350E84E12000000EC
:0C0C800000D000D000D0E82EFAD71200FF
:020C8C00120054
:00000001FF
